:0200000480007A
:100000006F000005732F2034930F80006308FF03F7
:10001000930F90006304FF03930FB0006300FF038E
:10002000130F000063040F0067000F00732F2034CC
:1000300063540F006F00400093E19153171F0000BD
:1000400023223FFC171F000023200FFC6FF01FFF2F
:100050009300000013010000930100001302000050
:100060009302000013030000930300001304000038
:100070009304000013050000930500001306000020
:100080009306000013070000930700001308000008
:10009000930800001309000093090000130A0000F0
:1000A000930A0000130B0000930B0000130C0000D8
:1000B000930C0000130D0000930D0000130E0000C0
:1000C000930E0000130F0000930F0000732540F102
:1000D0006310050097020000938202017390523072
:1000E000735044749702000093820201739052305F
:1000F00073500018970200009382420273905230AE
:100100009B021000939252039382F2FF7390023B82
:100110009302F0017390023A73504030970200004E
:1001200093824201739052307350203073503030BC
:100130009301000097020000938202ED7390523009
:10014000130510001315F501635C05000F00F00F97
:10015000930110009308D005130500007300000000
:1001600093020000638A020073905210B7B200003D
:100170009B829210739022307350003097020000DF
:100180009382420173901234732540F17300203042
:1001900093012000B707FF009B87F70F9397070194
:1001A0009387F70F939707019387F70F9720000026
:1001B000938040E503B70000B703FF009B83F30F74
:1001C000939303019383F30F939303019383F30FAB
:1001D0006316774693013000B70701FF9B8717F03E
:1001E00093970701938717F093970701938707F079
:1001F00097200000938000E103B78000B70301FF60
:100200009B8313F093930301938313F09393030160
:10021000938303F06314774293014000B707010012
:100220009B8717F093970701938717F09397070120
:10023000938717F09397C700938707FF97200000D5
:10024000938040DC03B70001B70301009B8313F0E8
:1002500093930301938313F093930301938313F018
:100260009393C300938303FF631A773C9301500079
:10027000B707FFFF9B87F70F939707019387F70F48
:10028000939707019387F70F9397C7009387F7001A
:1002900097200000938000D703B78001B703FFFFCA
:1002A0009B83F30F939303019383F30F93930301C2
:1002B0009383F30F9393C3009383F3006310773812
:1002C00093016000B707FF009B87F70F9397070123
:1002D0009387F70F939707019387F70F97200000F5
:1002E0009380C0D303B780FEB703FF009B83F30F57
:1002F000939303019383F30F939303019383F30F7A
:10030000631E773293017000B70701FF9B8717F0D8
:1003100093970701938717F093970701938707F047
:1003200097200000938080CF03B700FFB70301FF41
:100330009B8313F093930301938313F0939303012F
:10034000938303F0631C772E93018000B7070100AD
:100350009B8717F093970701938717F093970701EF
:10036000938717F09397C700938707FF97200000A4
:100370009380C0CA03B780FFB70301009B8313F0CB
:1003800093930301938313F093930301938313F0E7
:100390009393C300938303FF6312772A9301900022
:1003A000B707FFFF9B87F70F939707019387F70F17
:1003B000939707019387F70F9397C7009387F700E9
:1003C00097200000938080C503B70000B703FFFFAC
:1003D0009B83F30F939303019383F30F9393030191
:1003E0009383F30F9393C3009383F30063187724ED
:1003F0009301A000972000009380C0C0938000FE6E
:1004000083B20002B703FF009B83F30F93930301B2
:100410009383F30F939303019383F30F63907222FB
:100420009301B000972000009380C0BD9380D0FF5F
:1004300083B2B000B70301FF9B8313F093930301D2
:10044000938313F093930301938303F06398721ED5
:100450009301C0001302000097200000938000BBAE
:1004600003B7800013030700B70301009B8313F059
:1004700093930301938313F093930301938313F0F6
:100480009393C300938303FF631A731A130212003A
:1004900093022000E31252FC9301D00013020000EB
:1004A00097200000938000B703B78000130000007E
:1004B00013030700B703FFFF9B83F30F939303011D
:1004C0009383F30F939303019383F30F9393C300E9
:1004D0009383F30063147316130212009302200037
:1004E000E31052FC9301E00013020000972000008B
:1004F000938040B103B78000130000001300000098
:1005000013030700B70301FF9B8313F093930301C9
:10051000938313F093930301938303F06310731297
:100520001302120093022000E31252FC9301F00028
:100530001302000097200000938040AD03B78000B5
:10054000B70301009B8313F093930301938313F08C
:1005500093930301938313F09393C300938303FF57
:10056000631E770C1302120093022000E31452FC66
:10057000930100011302000097200000938080A9DE
:100580001300000003B78000B703FFFF9B83F30F46
:10059000939303019383F30F939303019383F30FD7
:1005A0009393C3009383F300631A77081302120036
:1005B00093022000E31252FC930110011302000089
:1005C00097200000938000A4130000001300000097
:1005D00003B78000B70301FF9B8313F093930301DC
:1005E000938313F093930301938303F063187704C9
:1005F0001302120093022000E31452FC9301200125
:1006000097220000938202A003B102001301200090
:1006100093032000631471029301300197220000BC
:100620009382429E03B102001300000013012000D8
:100630009303200063147100631030020F00F00F69
:10064000638001009391110093E111009308D0059C
:1006500013850100730000000F00F00F93011000DC
:100660009308D0051305000073000000731000C04C
:0C0670000000000000000000000000007E
:1010000000000000000000000000000000000000E0
:1010100000000000000000000000000000000000D0
:1010200000000000000000000000000000000000C0
:1010300000000000000000000000000000000000B0
:081040000000000000000000A8
:10200000FF00FF00FF00FF0000FF00FF00FF00FFD8
:10201000F00FF00FF00FF00F0FF00FF00FF00FF0C8
:040000058000000077
:00000001FF
